:0A04F00000010202030304040505E5
:10031900E4F513F512F511F510C203C200C202C2C9
:10032900011206B87E057F008E238F24752B057573
:100339002C1275210575221C752905752A3C752D08
:1003490005752E5C90E680E030E70E852125852233
:1003590026852927852A28800C852925852A268509
:100369002127852228EE54E0700302048A751400BF
:100379007515807E057F008E168F17C374E89FFF61
:1003890074059ECF2402CF3400FEE48F0F8E0EF544
:100399000DF50CF50BF50AF509F508AF0FAE0EAD25
:1003A9000DAC0CAB0BAA0AA909A808C3120D4D5034
:1003B9002AE515250BF582E514350AF58374CDF088
:1003C900E4FAF9F8E50B2401F50BEA350AF50AE92F
:1003D9003509F509E83508F50880C0E4F50BF50A93
:1003E900F509F508AF0FAE0EAD0DAC0CAB0BAA0AB3
:1003F900A909A808C3120D4D5035AE0AAF0BE51770
:100409002FF582E5163EF583E0FDE5152FF582E52A
:10041900143EF583EDF0E4FAF9F8EF2401F50BEA5F
:100429003EF50AE93509F509E83508F50880B58585
:10043900142385152474002480FF740534FFFEC33A
:10044900E52C9FF52CE52B9EF52BC3E5269FF5267C
:10045900E5259EF525C3E5289FF528E5279EF5277F
:10046900C3E5229FF522E5219EF521C3E52A9FF5E3
:100479002AE5299EF529C3E52E9FF52EE52D9EF542
:100489002DD2E843D82090E668E04409F090E65C74
:10049900E0443DF0D2AF90E680E020E105D20612BB
:1004A9000BDD90E680E054F7F0538EF8C20330017B
:1004B90005120080C2013003291204FE5024C20330
:1004C900120C6420001690E682E030E704E020E197
:1004D900EF90E682E030E604E020E0E4120C0C1232
:0704E90008F81209B880C7F2
:1000800090E6B9E0700302015B14700302020424DD
:10009000FE700302029924FB7003020155147003E1
:1000A00002014F147003020143147003020149243A
:1000B0000560030203051208FA400302031190E6EB
:1000C000BBE024FE602C14604724FD6016146031F0
:1000D00024067065E52390E6B3F0E52490E6B4F0DD
:1000E000020311E52B90E6B3F0E52C90E6B4F002A4
:1000F0000311E52590E6B3F0E52690E6B4F002039F
:1001000011E52790E6B3F0E52890E6B4F00203117C
:1001100090E6BAE0FF120C38AA06A9077B01EA496B
:10012000600DEE90E6B3F0EF90E6B4F002031190AC
:10013000E6A0E04401F002031190E6A0E04401F0E3
:10014000020311120D3B0203111208F002031112F7
:100150000B2D020311120D290203111208FC40039A
:1001600002031190E6B8E0247F602B14603C240267
:1001700060030201FAA200E433FF25E0FFA202E4DB
:10018000334F90E740F0E4A3F090E68AF090E68BDE
:100190007402F0020311E490E740F0A3F090E68AC5
:1001A000F090E68B7402F002031190E6BCE0547EFE
:1001B000FF7E00E0D3948040067C007D0180047CBB
:1001C000007D00EC4EFEED4F24F0F58274043EF508
:1001D00083E493FF3395E0FEEF24A1FFEE34E68F36
:1001E00082F583E0540190E740F0E4A3F090E68AC2
:1001F000F090E68B7402F002031190E6A0E0440157
:10020000F00203111208FE400302031190E6B8E069
:1002100024FE601D2402600302031190E6BAE0B4DC
:100220000105C20002031190E6A0E04401F00203C0
:100230001190E6BAE0705990E6BCE0547EFF7E0073
:10024000E0D3948040067C007D0180047C007D002A
:10025000EC4EFEED4F24F0F58274043EF583E493FA
:10026000FF3395E0FEEF24A1FFEE34E68F82F583A5
:10027000E054FEF090E6BCE05480FF131313541FCB
:10028000FFE0540F2F90E683F0E04420F0020311CA
:1002900090E6A0E04401F08078120D5E507390E685
:1002A000B8E024FE60202402706790E6BAE0B40152
:1002B00004D200805C90E6BAE06402605490E6A04C
:1002C000E04401F0804B90E6BCE0547EFF7E00E00D
:1002D000D3948040067C007D0180047C007D00EC8E
:1002E0004EFEED4F24F0F58274043EF583E493FF57
:1002F0003395E0FEEF24A1FFEE34E68F82F583E034
:100300004401F0800C1205EA500790E6A0E0440199
:08031000F090E6A0E04480F04B
:0103180022C2
:030033000204FACA
:0404FA0053D8EF32B2
:100500001201000200000040470502100000010235
:1005100000010A060002000000400100090220005C
:1005200001010080320904000002FF0000000705FD
:1005300002020002000705860200020009022000F4
:1005400001010080320904000002FF0000000705DD
:10055000020240000007058602400000040309046F
:10056000100343007900700072006500730073008F
:10057000780345005A002D0055005300420020002A
:100580004600580032002000470050004900460055
:10059000200074006F0020004500780074002000E7
:1005A0004600490046004F002000450078006100E9
:1005B0006D0070006C00650020007500730069001C
:1005C0006E00670020004600490046004F002000F2
:1005D0005400720061006E007300610063007400DB
:0A05E00069006F006E007300000058
:04083500C104C10534
:1006B80090E600E054E74410F000000090E6127461
:1006C800A0F0000000E490E613F000000090E614AB
:1006D80074E0F0000000E490E615F000000090E6F9
:1006E800047480F00000007402F00000007406F04A
:1006F800000000E4F000000090E61804F00000009C
:100708007411F000000090E61A7409F0000000125D
:10071800077900000090E6D27401F000000090E62E
:10072800E204F000000090109AE090E6C7F00000A4
:100738000090109DE090E6CBF00000009010A1E042
:1007480090E60CF000000090109FE090E6CCF000DE
:1007580000009010A0E090E6CDF000000043B20445
:100768004380045380FB7F017E00120AEC4380041F
:01077800225E
:1009B800E5BB30E74DE5AB20E14890E6F4E030E1F7
:1009C8004130051600000090E6D07401F0000000E8
:1009D800E490E6D1F00000008014000000E490E606
:1009E800D0F000000090E6D17420F0000000120C56
:1009F800AB000000E4F5BB000000E5BB30E7FB00FE
:100A08000000300452E5BB30E74D90E6F4E030E0FA
:100A180046E5AC20E04130051600000090E6D074B1
:100A280001F0000000E490E6D1F00000008014001E
:100A38000000E490E6D0F000000090E6D17420F0C9
:100A4800000000120C8900000075BB06000000E5DC
:080A5800BB30E7FB00000022A7
:0204FE00D32207
:0208F800D32209
:0208FA00D32207
:100B2D0090E680E030E71800000090E6247402F0B3
:100B3D00000000E490E625F0000000D205801600CC
:100B4D000000E490E624F000000090E6257440F0EB
:0D0B5D00000000C20590E6BAE0F51BD322AF
:100D290090E740E51BF0E490E68AF090E68B04F04A
:020D3900D322C3
:0808F00090E6BAE0F51AD322EC
:100D3B0090E740E51AF0E490E68AF090E68B04F039
:020D4B00D322B1
:0208FC00D32205
:0208FE00D32203
:020D5E00D3229E
:1005EA0090E6B9E0244D60401460581460701470AD
:1005FA0003020690240460030206B443B204438053
:10060A00045380FB7F017E00120AEC43800490E7CA
:10061A004074B2F0E490E68AF090E68B04F090E63B
:10062A00A0E04480F00206B6D20490E74074B3F02A
:10063A00E490E68AF090E68B04F090E6A0E044802D
:10064A00F08069C20490E74074B4F0E490E68AF05E
:10065A0090E68B04F090E6A0E04480F0804E90E7AC
:10066A004074B5F000000090E6F4E090E741F00035
:10067A000000E490E68AF090E68B7402F090E6A01F
:10068A00E04480F0802690E74074B6F0000000A3B2
:10069A00E5BBF0000000E490E68AF090E68B740275
:0E06AA00F090E6A0E04480F08002D322C3224C
:100CCD00C0E0C083C082D2015391EF90E65D740104
:080CDD00F0D082D083D0E03298
:100CFD00C0E0C083C0825391EF90E65D7404F0D0E4
:060D0D0082D083D0E03229
:100D1300C0E0C083C0825391EF90E65D7402F0D0CF
:060D230082D083D0E03213
:100BA700C0E0C083C082852925852A2685268285BF
:100BB7002583A37402F0852127852228852882852D
:100BC7002783A37407F05391EF90E65D7410F0D07C
:060BD70082D083D0E03261
:100CE500C0E0C083C082D2035391EF90E65D7408E3
:080CF500F0D082D083D0E03280
:100B6A00C0E0C083C08290E680E030E7208521257E
:100B7A00852226852682852583A37402F085292766
:100B8A00852A28852882852783A37407F05391EF45
:0D0B9A0090E65D7420F0D082D083D0E03270
:010D60003260
:010D6100325F
:010D6200325E
:010D6300325D
:010D6400325C
:010D6500325B
:010D6600325A
:010D67003259
:010D68003258
:010D69003257
:010D6A003256
:010D6B003255
:010D6C003254
:010D6D003253
:010D6E003252
:010D6F003251
:010D70003250
:010D7100324F
:010D7200324E
:010D7300324D
:010D7400324C
:010D7500324B
:010D7600324A
:010D77003249
:010D78003248
:010D79003247
:010D7A003246
:010D7B003245
:010D7C003244
:010D7D003243
:010D7E003242
:010D7F003241
:010D80003240
:010D8100323F
:010D8200323E
:010D8300323D
:100C8900901099E090E6C6F000000090109BE0906B
:100C9900E6C8F000000090109CE090E6C9F0000062
:020CA900002227
:100CAB009010A2E090E6C6F00000009010A4E09037
:100CBB00E6C8F00000009010A5E090E6C9F0000037
:020CCB00002205
:100C0C0090E682E030E004E020E60B90E682E030F3
:100C1C00E119E030E71590E680E04401F07F147EA6
:0C0C2C0000120AEC90E680E054FEF0227A
:100C640090E682E044C0F090E681F0438701000002
:040C7400000000225A
:100BDD0030060990E680E0440AF0800790E680E058
:100BED004408F07FDC7E05120AEC90E65D74FFF0A0
:0F0BFD0090E65FF05391EF90E680E054F7F0221E
:100AEC008E188F1990E600E05418700DE518C3139A
:100AFC00F518E51913F519801590E600E05418FF68
:100B0C00BF100BE51925E0F519E51833F518E519B3
:100B1C001519AE18700215184E6005120C7880EE7F
:010B2C0022A6
:020C3800A9070A
:100C3A00AE2DAF2E8F828E83A3E064037017AD01B1
:100C4A0019ED7001228F828E83E07C002FFDEC3E2D
:090C5A00FEAF0580DF7E007F0083
:010C6300226E
:100C78007400F58690FDA57C05A3E582458370F98F
:010C88002249
:03004300020900AF
:030053000209009F
:10090000020CCD00020D1300020CFD00020CE500EC
:10091000020BA700020B6A00020D6000020D6100CD
:10092000020D6200020D6300020D6400020D6500FD
:10093000020D6600020D6700020D6800020D6900DD
:10094000020D6A00020D6100020D6B00020D6C00C9
:10095000020D6D00020D6E00020D6F00020D7000A1
:10096000020D7100020D6100020D6100020D6100B7
:10097000020D7200020D7300020D7400020D75006D
:10098000020D7600020D7700020D7800020D79004D
:10099000020D7A00020D7B00020D7C00020D7D002D
:1009A000020D7E00020D7F00020D8000020D81000D
:0809B000020D8200020D83001C
:1008390060801000010101010101010700000000B1
:100849000000000007070707070707070000000067
:100859000000003F01010101010101070000000042
:100869000000000007070707070707070000000047
:100879000000003F0101013B0101010700000003E5
:100889000202020007050107070707070000002DFC
:100899000000003F013901010101010700030202C3
:1008A900020202000707070707070707002D0000D4
:1008B9000000003F602410870000000000000000D5
:1008C900000000000000000000008336010704005A
:1008D900030201813606070400030200471080E085
:0608E900000007EE4E00C6
:1007790090E60174EEF090E6F574FFF0901080E0D9
:1007890090E6F3F0901081E090E6C3F0901082E0DB
:1007990090E6C1F0901083E090E6C2F0901085E0F9
:1007A90090E6C0F0901086E090E6F4F075AF07741B
:1007B90010F59A7400F59B759DE4E4F59EFF90E6AB
:1007C9007BE090E67CF00FBF80F490E67174FFF057
:1007D900F5B490E672E04480F043B680000000E48E
:1007E90090E6C4F000000090E6C5F0901087E09014
:1007F900E6C6F0901088E090E6C7F0901089E09086
:10080900E6C8F090108AE090E6C9F090108BE0906D
:10081900E6CAF090108CE090E6CBF090108DE09055
:0B082900E6CCF090108EE090E6CDF0E1
:0108340022A1
:03000000020A6091
:0C0A6000787FE4F6D8FD75812E020AA70D
:100D4D00EB9FF5F0EA9E42F0E99D42F0E89C45F0FC
:010D5D002273
:100A6C00020319E493A3F8E493A34003F68001F284
:100A7C0008DFF48029E493A3F85407240CC8C3338B
:100A8C00C4540F4420C8834004F456800146F6DF5A
:100A9C00E4800B0102040810204080900835E47EAD
:100AAC00019360BCA3FF543F30E509541FFEE4934F
:100ABC00A360010ECF54C025E060A840B8E493A316
:100ACC00FAE493A3F8E493A3C8C582C8CAC583CA41
:100ADC00F0A3C8C582C8CAC583CADFE9DEE780BEF9
:0108EF000008
:00000001FF
